******************************************************************************
                  TI ARM Linker Unix v18.1.2                   
******************************************************************************
>> Linked Tue Jun 19 13:32:45 2018

OUTPUT FILE NAME:   <Led_blink_FreeRTOS.out>
ENTRY POINT SYMBOL: "_c_int00_noargs"  address: 200076c9


MEMORY CONFIGURATION

         name            origin    length      used     unused   attr    fill
----------------------  --------  ---------  --------  --------  ----  --------
  SRAM_CODE             20004000   00012fff  00003b62  0000f49d  RW X
  SRAM_DATA             20017000   00019000  0000428f  00014d71  RW X


SEGMENT ALLOCATION MAP

run origin  load origin   length   init length attrs members
----------  ----------- ---------- ----------- ----- -------
20004000    20004000    00003b68   00003b68    r-x
  20004000    20004000    00000400   00000400    r-- .intvecs
  20004400    20004400    0000345e   0000345e    r-x .text
  20007860    20007860    000002ac   000002ac    r-- .const
  20007b10    20007b10    00000058   00000058    r-- .cinit
20017000    20017000    00002248   00000000    rw-
  20017000    20017000    00002048   00000000    rw- .sysmem
  20019048    20019048    00000187   00000000    rw- .bss
  200191d0    200191d0    00000078   00000000    rw- .data
2002dfb8    2002dfb8    00002048   00000000    rw-
  2002dfb8    2002dfb8    00002048   00000000    rw- .stack


SECTION ALLOCATION MAP

 output                                  attributes/
section   page    origin      length       input sections
--------  ----  ----------  ----------   ----------------
.intvecs   0    20004000    00000400     
                  20004000    00000400     startup_ccs.obj (.intvecs)

.init_array 
*          0    20004000    00000000     UNINITIALIZED

.text      0    20004400    0000345e     
                  20004400    0000125c     free_rtos.a : tasks.obj (.text)
                  2000565c    00000b24                 : queue.obj (.text)
                  20006180    0000045c                 : osi_freertos.obj (.text)
                  200065dc    00000390     gpio_if.obj (.text)
                  2000696c    00000178     driverlib.a : prcm.obj (.text:PRCMCC3200MCUInit)
                  20006ae4    0000012a     free_rtos.a : list.obj (.text)
                  20006c0e    00000002     driverlib.a : interrupt.obj (.text:IntDefaultHandler)
                  20006c10    00000110     free_rtos.a : port.obj (.text)
                  20006d20    000000d8     rtsv7M4_T_le_eabi.lib : memory.c.obj (.text:free)
                  20006df8    000000ba     free_rtos.a : portasm.obj (.text)
                  20006eb2    00000002     rtsv7M4_T_le_eabi.lib : _lock.c.obj (.text:_nop)
                  20006eb4    000000a8     driverlib.a : interrupt.obj (.text:IntDisable)
                  20006f5c    000000a8                 : interrupt.obj (.text:IntEnable)
                  20007004    000000a4     main.obj (.text)
                  200070a8    0000009c     rtsv7M4_T_le_eabi.lib : memcpy_t2.asm.obj (.text)
                  20007144    00000088     driverlib.a : pin.obj (.text:PinConfigSet)
                  200071cc    00000082                 : gpio.obj (.text:GPIOIntTypeSet)
                  2000724e    0000007a     rtsv7M4_T_le_eabi.lib : memset_t2.asm.obj (.text)
                  200072c8    00000078                           : memory.c.obj (.text:malloc)
                  20007340    00000068                           : copy_decompress_lzss.c.obj (.text:decompress:lzss:__TI_decompress_lzss)
                  200073a8    00000058     driverlib.a : prcm.obj (.text:PRCMPeripheralReset)
                  20007400    00000054                 : interrupt.obj (.text:IntPrioritySet)
                  20007454    0000004c     pinmux.obj (.text)
                  200074a0    00000044     rtsv7M4_T_le_eabi.lib : autoinit.c.obj (.text:__TI_auto_init_nobinit_nopinit:__TI_auto_init_nobinit_nopinit)
                  200074e4    00000040     driverlib.a : pin.obj (.text:PinModeSet)
                  20007524    0000003c                 : prcm.obj (.text:PRCMPeripheralClkEnable)
                  20007560    0000003c     rtsv7M4_T_le_eabi.lib : memory.c.obj (.text:minsert)
                  2000759c    00000038     free_rtos.a : heap_3.obj (.text)
                  200075d4    00000038     rtsv7M4_T_le_eabi.lib : memory.c.obj (.text:minit)
                  2000760c    00000036     driverlib.a : gpio.obj (.text:GPIODirModeSet)
                  20007642    00000030                 : pin.obj (.text:PinTypeGPIO)
                  20007672    00000002     --HOLE-- [fill = 0]
                  20007674    0000002c                 : prcm.obj (.text:PRCMSysResetCauseGet)
                  200076a0    00000028                 : prcm.obj (.text:PRCMPeripheralClkDisable)
                  200076c8    00000028     rtsv7M4_T_le_eabi.lib : boot_cortex_m.c.obj (.text:_c_int00_noargs:_c_int00_noargs)
                  200076f0    00000028                           : memory.c.obj (.text:mremove)
                  20007718    00000024     driverlib.a : interrupt.obj (.text:IntUnregister)
                  2000773c    00000020                 : gpio.obj (.text:GPIOPinWrite)
                  2000775c    00000020                 : interrupt.obj (.text:IntRegister)
                  2000777c    0000001a                 : gpio.obj (.text:GPIOIntEnable)
                  20007796    00000018                 : gpio.obj (.text:GPIOPinRead)
                  200077ae    00000016                 : prcm.obj (.text:PRCMHIBRegRead)
                  200077c4    00000016                 : prcm.obj (.text:PRCMHIBRegWrite)
                  200077da    00000014                 : cpu.obj (.text:CPUcpsie)
                  200077ee    00000014                 : gpio.obj (.text:GPIOIntClear)
                  20007802    00000002     --HOLE-- [fill = 0]
                  20007804    00000014                 : interrupt.obj (.text:IntVTableBaseSet)
                  20007818    00000012     rtsv7M4_T_le_eabi.lib : copy_zero_init.c.obj (.text:decompress:ZI:__TI_zero_init_nomemset:__TI_zero_init_nomemset)
                  2000782a    0000000e                           : copy_decompress_none.c.obj (.text:decompress:none:__TI_decompress_none)
                  20007838    0000000e     startup_ccs.obj (.text)
                  20007846    0000000a     driverlib.a : interrupt.obj (.text:IntMasterEnable)
                  20007850    00000006                 : utils.obj (.text:UtilsDelay)
                  20007856    00000004     rtsv7M4_T_le_eabi.lib : pre_init.c.obj (.text:_system_pre_init)
                  2000785a    00000004                           : exit.c.obj (.text:abort:abort)

.const     0    20007860    000002ac     
                  20007860    00000100     driverlib.a : pin.obj (.const:g_ulPinToPadMap)
                  20007960    000000d4                 : interrupt.obj (.const:g_pulRegs)
                  20007a34    000000a8                 : prcm.obj (.const:PRCM_PeriphRegsList)
                  20007adc    00000018                 : interrupt.obj (.const:g_pulDisRegs)
                  20007af4    00000018                 : interrupt.obj (.const:g_pulEnRegs)

.cinit     0    20007b10    00000058     
                  20007b10    00000032     (.cinit..data.load) [load image, compression = lzss]
                  20007b42    00000002     --HOLE-- [fill = 0]
                  20007b44    0000000c     (__TI_handler_table)
                  20007b50    00000008     (.cinit..bss.load) [load image, compression = zero_init]
                  20007b58    00000010     (__TI_cinit_table)

.sysmem    0    20017000    00002048     UNINITIALIZED
                  20017000    00000008     rtsv7M4_T_le_eabi.lib : memory.c.obj (.sysmem)
                  20017008    00002040     --HOLE--

.bss       0    20019048    00000187     UNINITIALIZED
                  20019048    000000c8     free_rtos.a : tasks.obj (.bss:pxReadyTasksLists)
                  20019110    00000050     (.common:xQueueRegistry)
                  20019160    00000014                 : tasks.obj (.bss:xDelayedTaskList1)
                  20019174    00000014                 : tasks.obj (.bss:xDelayedTaskList2)
                  20019188    00000014                 : tasks.obj (.bss:xPendingReadyList)
                  2001919c    00000014                 : tasks.obj (.bss:xSuspendedTaskList)
                  200191b0    00000014                 : tasks.obj (.bss:xTasksWaitingTermination)
                  200191c4    00000008                 : tasks.obj (.bss)
                  200191cc    00000001     (.common:g_ucLED1Pin)
                  200191cd    00000001     (.common:g_ucLED2Pin)
                  200191ce    00000001     (.common:g_ucLED3Pin)

.data      0    200191d0    00000078     UNINITIALIZED
                  200191d0    00000034     free_rtos.a : tasks.obj (.data)
                  20019204    00000014     gpio_if.obj (.data:ulReg)
                  20019218    0000000c     rtsv7M4_T_le_eabi.lib : memory.c.obj (.data:$O1$$)
                  20019224    0000000c     free_rtos.a : osi_freertos.obj (.data)
                  20019230    0000000c     gpio_if.obj (.data)
                  2001923c    00000008     rtsv7M4_T_le_eabi.lib : _lock.c.obj (.data:$O1$$)
                  20019244    00000004     free_rtos.a : port.obj (.data)

.stack     0    2002dfb8    00002048     UNINITIALIZED
                  2002dfb8    00000004     rtsv7M4_T_le_eabi.lib : boot_cortex_m.c.obj (.stack)
                  2002dfbc    00002044     --HOLE--

MODULE SUMMARY

       Module                       code    ro data   rw data
       ------                       ----    -------   -------
    ./
       startup_ccs.obj              14      1024      0      
       gpio_if.obj                  912     0         35     
       main.obj                     164     0         0      
       pinmux.obj                   76      0         0      
    +--+----------------------------+-------+---------+---------+
       Total:                       1166    1024      35     
                                                             
    /home/nirmal/ti/ccsv8/tools/compiler/ti-cgt-arm_18.1.2.LTS/lib/rtsv7M4_T_le_eabi.lib
       memory.c.obj                 492     0         12     
       memcpy_t2.asm.obj            156     0         0      
       memset_t2.asm.obj            122     0         0      
       copy_decompress_lzss.c.obj   104     0         0      
       autoinit.c.obj               68      0         0      
       boot_cortex_m.c.obj          40      0         0      
       copy_zero_init.c.obj         18      0         0      
       copy_decompress_none.c.obj   14      0         0      
       _lock.c.obj                  2       0         8      
       exit.c.obj                   4       0         0      
       pre_init.c.obj               4       0         0      
    +--+----------------------------+-------+---------+---------+
       Total:                       1024    0         20     
                                                             
    /home/nirmal/ti/sdks/cc3200-sdk/driverlib/ccs/Release/driverlib.a
       prcm.obj                     652     168       0      
       interrupt.obj                520     260       0      
       pin.obj                      248     256       0      
       gpio.obj                     286     0         0      
       cpu.obj                      20      0         0      
       utils.obj                    6       0         0      
    +--+----------------------------+-------+---------+---------+
       Total:                       1732    684       0      
                                                             
    /home/nirmal/ti/sdks/cc3200-sdk/oslib/ccs/free_rtos/free_rtos.a
       tasks.obj                    4700    0         360    
       queue.obj                    2852    0         80     
       osi_freertos.obj             1116    0         12     
       list.obj                     298     0         0      
       port.obj                     272     0         4      
       portasm.obj                  186     0         0      
       heap_3.obj                   56      0         0      
    +--+----------------------------+-------+---------+---------+
       Total:                       9480    0         456    
                                                             
       Heap:                        0       0         8264   
       Stack:                       0       0         8264   
       Linker Generated:            0       86        0      
    +--+----------------------------+-------+---------+---------+
       Grand Total:                 13402   1794      17039  


LINKER GENERATED COPY TABLES

__TI_cinit_table @ 20007b58 records: 2, size/record: 8, table size: 16
	.data: load addr=20007b10, load size=00000032 bytes, run addr=200191d0, run size=00000078 bytes, compression=lzss
	.bss: load addr=20007b50, load size=00000008 bytes, run addr=20019048, run size=00000187 bytes, compression=zero_init


LINKER GENERATED HANDLER TABLE

__TI_handler_table @ 20007b44 records: 3, size/record: 4, table size: 12
	index: 0, handler: __TI_decompress_lzss
	index: 1, handler: __TI_decompress_none
	index: 2, handler: __TI_zero_init


GLOBAL SYMBOLS: SORTED ALPHABETICALLY BY Name 

address   name                             
-------   ----                             
2000785b  C$$EXIT                          
200077db  CPUcpsie                         
2000760d  GPIODirModeSet                   
200077ef  GPIOIntClear                     
2000777d  GPIOIntEnable                    
200071cd  GPIOIntTypeSet                   
20007797  GPIOPinRead                      
2000773d  GPIOPinWrite                     
2000689d  GPIO_IF_ConfigureNIntEnable      
20006919  GPIO_IF_Get                      
20006857  GPIO_IF_GetPortNPin              
20006619  GPIO_IF_LedConfigure             
2000670b  GPIO_IF_LedOff                   
20006657  GPIO_IF_LedOn                    
200067bf  GPIO_IF_LedStatus                
20006829  GPIO_IF_LedToggle                
200068df  GPIO_IF_Set                      
20006eb5  IntDisable                       
20006f5d  IntEnable                        
20007847  IntMasterEnable                  
20007401  IntPrioritySet                   
2000775d  IntRegister                      
20007719  IntUnregister                    
20007805  IntVTableBaseSet                 
2000696d  PRCMCC3200MCUInit                
200077af  PRCMHIBRegRead                   
200077c5  PRCMHIBRegWrite                  
200076a1  PRCMPeripheralClkDisable         
20007525  PRCMPeripheralClkEnable          
200073a9  PRCMPeripheralReset              
20007675  PRCMSysResetCauseGet             
20007145  PinConfigSet                     
200074e5  PinModeSet                       
20007455  PinMuxConfig                     
20007643  PinTypeGPIO                      
20007839  ResetISR                         
20007851  UtilsDelay                       
20006449  VDeleteSimpleLinkSpawnTask       
200063f9  VStartSimpleLinkSpawnTask        
20030000  __STACK_END                      
00002048  __STACK_SIZE                     
00002048  __SYSMEM_SIZE                    
20007b58  __TI_CINIT_Base                  
20007b68  __TI_CINIT_Limit                 
20007b44  __TI_Handler_Table_Base          
20007b50  __TI_Handler_Table_Limit         
200074a1  __TI_auto_init_nobinit_nopinit   
20007341  __TI_decompress_lzss             
2000782b  __TI_decompress_none             
ffffffff  __TI_pprof_out_hndl              
ffffffff  __TI_prof_data_size              
ffffffff  __TI_prof_data_start             
20007b10  __TI_static_base__               
20007819  __TI_zero_init_nomemset          
2000724f  __aeabi_memclr                   
2000724f  __aeabi_memclr4                  
2000724f  __aeabi_memclr8                  
200070a9  __aeabi_memcpy                   
200070a9  __aeabi_memcpy4                  
200070a9  __aeabi_memcpy8                  
20007251  __aeabi_memset                   
20007251  __aeabi_memset4                  
20007251  __aeabi_memset8                  
ffffffff  __binit__                        
ffffffff  __c_args__                       
UNDEFED   __mpu_init                       
2002dfb8  __stack                          
200076c9  _c_int00_noargs                  
2001923c  _lock                            
20006eb3  _nop                             
20017000  _sys_memory                      
UNDEFED   _system_post_cinit               
20007857  _system_pre_init                 
20019240  _unlock                          
2000785b  abort                            
ffffffff  binit                            
20004691  eTaskGetState                    
20006d21  free                             
20004000  g_pfnVectors                     
200191cc  g_ucLED1Pin                      
200191cd  g_ucLED2Pin                      
200191ce  g_ucLED3Pin                      
20019230  g_uiLED1Port                     
20019234  g_uiLED2Port                     
20019238  g_uiLED3Port                     
20007053  main                             
200072c9  malloc                           
2000654d  mem_Free                         
20006541  mem_Malloc                       
2000656d  mem_copy                         
20006559  mem_set                          
200070a9  memcpy                           
20007257  memset                           
200075d5  minit                            
200065c3  osi_ContextRestore               
200065c1  osi_ContextSave                  
20006581  osi_EnterCritical                
2000658b  osi_ExitCritical                 
200061a7  osi_InterruptDeRegister          
20006181  osi_InterruptRegister            
200062b1  osi_LockObjCreate                
20006325  osi_LockObjDelete                
20006335  osi_LockObjLock                  
20006361  osi_LockObjUnlock                
20006475  osi_MsgQCreate                   
200064b9  osi_MsgQDelete                   
20006505  osi_MsgQRead                     
200064d3  osi_MsgQWrite                    
2000659d  osi_Sleep                        
2000638b  osi_Spawn                        
2000628f  osi_SyncObjClear                 
200061b9  osi_SyncObjCreate                
200061e9  osi_SyncObjDelete                
20006203  osi_SyncObjSignal                
2000622b  osi_SyncObjSignalFromISR         
20006263  osi_SyncObjWait                  
200062d7  osi_TaskCreate                   
20006317  osi_TaskDelete                   
200065ad  osi_TaskDisable                  
200065b7  osi_TaskEnable                   
20006595  osi_start                        
20004bb5  pcTaskGetTaskName                
20006ead  portCLZ                          
20006e95  prvPortStartFirstTask            
2000759d  pvPortMalloc                     
200191d0  pxCurrentTCB                     
20006c11  pxPortInitialiseStack            
20005ddd  ucQueueGetQueueType              
20006dfd  ulPortSetInterruptMask           
20006bc7  uxListRemove                     
20005dbd  uxQueueGetQueueNumber            
20005d51  uxQueueMessagesWaiting           
20005d87  uxQueueMessagesWaitingFromISR    
20005d67  uxQueueSpacesAvailable           
20004ba9  uxTaskGetNumberOfTasks           
20004bd9  uxTaskGetSystemState             
200050cd  uxTaskGetTaskNumber              
20004725  uxTaskPriorityGet                
20005625  uxTaskResetEventItemValue        
20007011  vApplicationIdleHook             
20007013  vApplicationMallocFailedHook     
20007015  vApplicationStackOverflowHook    
20007005  vAssertCalled                    
20006ae5  vListInitialise                  
20006b15  vListInitialiseItem              
20006b61  vListInsert                      
20006b25  vListInsertEnd                   
20006e13  vPortClearInterruptMask          
20006c8d  vPortEndScheduler                
20006ca1  vPortEnterCritical               
20006cb9  vPortExitCritical                
200075bd  vPortFree                        
20006e6d  vPortSVCHandler                  
20006ced  vPortSetupTimerInterrupt         
20006c8f  vPortYield                       
20005ff7  vQueueAddToRegistry              
20005d99  vQueueDelete                     
20005dcb  vQueueSetQueueNumber             
20006039  vQueueUnregisterQueue            
2000463b  vTaskDelay                       
2000459f  vTaskDelayUntil                  
2000450f  vTaskDelete                      
20004a8d  vTaskEndScheduler                
200050bf  vTaskMissedYield                 
20004e55  vTaskPlaceOnEventList            
20004eb9  vTaskPlaceOnUnorderedEventList   
2000559b  vTaskPriorityDisinherit          
200054e1  vTaskPriorityInherit             
2000475d  vTaskPrioritySet                 
20004955  vTaskResume                      
200050ed  vTaskSetTaskNumber               
2000501f  vTaskSetTimeOutState             
20004a43  vTaskStartScheduler              
20004861  vTaskSuspend                     
20004a9f  vTaskSuspendAll                  
20004dd5  vTaskSwitchContext               
20019224  xHigherPriorityTaskWoken         
20006e21  xPortPendSVHandler               
20006c61  xPortStartScheduler              
20006cd1  xPortSysTickHandler              
20006087  xQueueAddToSet                   
200059b9  xQueueAltGenericReceive          
2000590d  xQueueAltGenericSend             
200057e1  xQueueCreateCountingSemaphore    
20005763  xQueueCreateMutex                
20006073  xQueueCreateSet                  
200056ed  xQueueGenericCreate              
20005b53  xQueueGenericReceive             
2000565d  xQueueGenericReset               
20005801  xQueueGenericSend                
20005ab7  xQueueGenericSendFromISR         
20005f93  xQueueIsQueueEmptyFromISR        
20005fd5  xQueueIsQueueFullFromISR         
20005d0d  xQueuePeekFromISR                
20005c95  xQueueReceiveFromISR             
20019110  xQueueRegistry                   
200060bb  xQueueRemoveFromSet              
200060fd  xQueueSelectFromSet              
20006117  xQueueSelectFromSetFromISR       
20019228  xSimpleLinkSpawnQueue            
2001922c  xSimpleLinkSpawnTaskHndl         
20005045  xTaskCheckForTimeOut             
20004401  xTaskGenericCreate               
20005495  xTaskGetCurrentTaskHandle        
20004c97  xTaskGetIdleTaskHandle           
200054a9  xTaskGetSchedulerState           
20004b7d  xTaskGetTickCount                
20004b91  xTaskGetTickCountFromISR         
20004cb1  xTaskIncrementTick               
20004f2d  xTaskRemoveFromEventList         
20004fb1  xTaskRemoveFromUnorderedEventList
20004ab1  xTaskResumeAll                   
200049c9  xTaskResumeFromISR               


GLOBAL SYMBOLS: SORTED BY Symbol Address 

address   name                             
-------   ----                             
00002048  __STACK_SIZE                     
00002048  __SYSMEM_SIZE                    
20004000  g_pfnVectors                     
20004401  xTaskGenericCreate               
2000450f  vTaskDelete                      
2000459f  vTaskDelayUntil                  
2000463b  vTaskDelay                       
20004691  eTaskGetState                    
20004725  uxTaskPriorityGet                
2000475d  vTaskPrioritySet                 
20004861  vTaskSuspend                     
20004955  vTaskResume                      
200049c9  xTaskResumeFromISR               
20004a43  vTaskStartScheduler              
20004a8d  vTaskEndScheduler                
20004a9f  vTaskSuspendAll                  
20004ab1  xTaskResumeAll                   
20004b7d  xTaskGetTickCount                
20004b91  xTaskGetTickCountFromISR         
20004ba9  uxTaskGetNumberOfTasks           
20004bb5  pcTaskGetTaskName                
20004bd9  uxTaskGetSystemState             
20004c97  xTaskGetIdleTaskHandle           
20004cb1  xTaskIncrementTick               
20004dd5  vTaskSwitchContext               
20004e55  vTaskPlaceOnEventList            
20004eb9  vTaskPlaceOnUnorderedEventList   
20004f2d  xTaskRemoveFromEventList         
20004fb1  xTaskRemoveFromUnorderedEventList
2000501f  vTaskSetTimeOutState             
20005045  xTaskCheckForTimeOut             
200050bf  vTaskMissedYield                 
200050cd  uxTaskGetTaskNumber              
200050ed  vTaskSetTaskNumber               
20005495  xTaskGetCurrentTaskHandle        
200054a9  xTaskGetSchedulerState           
200054e1  vTaskPriorityInherit             
2000559b  vTaskPriorityDisinherit          
20005625  uxTaskResetEventItemValue        
2000565d  xQueueGenericReset               
200056ed  xQueueGenericCreate              
20005763  xQueueCreateMutex                
200057e1  xQueueCreateCountingSemaphore    
20005801  xQueueGenericSend                
2000590d  xQueueAltGenericSend             
200059b9  xQueueAltGenericReceive          
20005ab7  xQueueGenericSendFromISR         
20005b53  xQueueGenericReceive             
20005c95  xQueueReceiveFromISR             
20005d0d  xQueuePeekFromISR                
20005d51  uxQueueMessagesWaiting           
20005d67  uxQueueSpacesAvailable           
20005d87  uxQueueMessagesWaitingFromISR    
20005d99  vQueueDelete                     
20005dbd  uxQueueGetQueueNumber            
20005dcb  vQueueSetQueueNumber             
20005ddd  ucQueueGetQueueType              
20005f93  xQueueIsQueueEmptyFromISR        
20005fd5  xQueueIsQueueFullFromISR         
20005ff7  vQueueAddToRegistry              
20006039  vQueueUnregisterQueue            
20006073  xQueueCreateSet                  
20006087  xQueueAddToSet                   
200060bb  xQueueRemoveFromSet              
200060fd  xQueueSelectFromSet              
20006117  xQueueSelectFromSetFromISR       
20006181  osi_InterruptRegister            
200061a7  osi_InterruptDeRegister          
200061b9  osi_SyncObjCreate                
200061e9  osi_SyncObjDelete                
20006203  osi_SyncObjSignal                
2000622b  osi_SyncObjSignalFromISR         
20006263  osi_SyncObjWait                  
2000628f  osi_SyncObjClear                 
200062b1  osi_LockObjCreate                
200062d7  osi_TaskCreate                   
20006317  osi_TaskDelete                   
20006325  osi_LockObjDelete                
20006335  osi_LockObjLock                  
20006361  osi_LockObjUnlock                
2000638b  osi_Spawn                        
200063f9  VStartSimpleLinkSpawnTask        
20006449  VDeleteSimpleLinkSpawnTask       
20006475  osi_MsgQCreate                   
200064b9  osi_MsgQDelete                   
200064d3  osi_MsgQWrite                    
20006505  osi_MsgQRead                     
20006541  mem_Malloc                       
2000654d  mem_Free                         
20006559  mem_set                          
2000656d  mem_copy                         
20006581  osi_EnterCritical                
2000658b  osi_ExitCritical                 
20006595  osi_start                        
2000659d  osi_Sleep                        
200065ad  osi_TaskDisable                  
200065b7  osi_TaskEnable                   
200065c1  osi_ContextSave                  
200065c3  osi_ContextRestore               
20006619  GPIO_IF_LedConfigure             
20006657  GPIO_IF_LedOn                    
2000670b  GPIO_IF_LedOff                   
200067bf  GPIO_IF_LedStatus                
20006829  GPIO_IF_LedToggle                
20006857  GPIO_IF_GetPortNPin              
2000689d  GPIO_IF_ConfigureNIntEnable      
200068df  GPIO_IF_Set                      
20006919  GPIO_IF_Get                      
2000696d  PRCMCC3200MCUInit                
20006ae5  vListInitialise                  
20006b15  vListInitialiseItem              
20006b25  vListInsertEnd                   
20006b61  vListInsert                      
20006bc7  uxListRemove                     
20006c11  pxPortInitialiseStack            
20006c61  xPortStartScheduler              
20006c8d  vPortEndScheduler                
20006c8f  vPortYield                       
20006ca1  vPortEnterCritical               
20006cb9  vPortExitCritical                
20006cd1  xPortSysTickHandler              
20006ced  vPortSetupTimerInterrupt         
20006d21  free                             
20006dfd  ulPortSetInterruptMask           
20006e13  vPortClearInterruptMask          
20006e21  xPortPendSVHandler               
20006e6d  vPortSVCHandler                  
20006e95  prvPortStartFirstTask            
20006ead  portCLZ                          
20006eb3  _nop                             
20006eb5  IntDisable                       
20006f5d  IntEnable                        
20007005  vAssertCalled                    
20007011  vApplicationIdleHook             
20007013  vApplicationMallocFailedHook     
20007015  vApplicationStackOverflowHook    
20007053  main                             
200070a9  __aeabi_memcpy                   
200070a9  __aeabi_memcpy4                  
200070a9  __aeabi_memcpy8                  
200070a9  memcpy                           
20007145  PinConfigSet                     
200071cd  GPIOIntTypeSet                   
2000724f  __aeabi_memclr                   
2000724f  __aeabi_memclr4                  
2000724f  __aeabi_memclr8                  
20007251  __aeabi_memset                   
20007251  __aeabi_memset4                  
20007251  __aeabi_memset8                  
20007257  memset                           
200072c9  malloc                           
20007341  __TI_decompress_lzss             
200073a9  PRCMPeripheralReset              
20007401  IntPrioritySet                   
20007455  PinMuxConfig                     
200074a1  __TI_auto_init_nobinit_nopinit   
200074e5  PinModeSet                       
20007525  PRCMPeripheralClkEnable          
2000759d  pvPortMalloc                     
200075bd  vPortFree                        
200075d5  minit                            
2000760d  GPIODirModeSet                   
20007643  PinTypeGPIO                      
20007675  PRCMSysResetCauseGet             
200076a1  PRCMPeripheralClkDisable         
200076c9  _c_int00_noargs                  
20007719  IntUnregister                    
2000773d  GPIOPinWrite                     
2000775d  IntRegister                      
2000777d  GPIOIntEnable                    
20007797  GPIOPinRead                      
200077af  PRCMHIBRegRead                   
200077c5  PRCMHIBRegWrite                  
200077db  CPUcpsie                         
200077ef  GPIOIntClear                     
20007805  IntVTableBaseSet                 
20007819  __TI_zero_init_nomemset          
2000782b  __TI_decompress_none             
20007839  ResetISR                         
20007847  IntMasterEnable                  
20007851  UtilsDelay                       
20007857  _system_pre_init                 
2000785b  C$$EXIT                          
2000785b  abort                            
20007b10  __TI_static_base__               
20007b44  __TI_Handler_Table_Base          
20007b50  __TI_Handler_Table_Limit         
20007b58  __TI_CINIT_Base                  
20007b68  __TI_CINIT_Limit                 
20017000  _sys_memory                      
20019110  xQueueRegistry                   
200191cc  g_ucLED1Pin                      
200191cd  g_ucLED2Pin                      
200191ce  g_ucLED3Pin                      
200191d0  pxCurrentTCB                     
20019224  xHigherPriorityTaskWoken         
20019228  xSimpleLinkSpawnQueue            
2001922c  xSimpleLinkSpawnTaskHndl         
20019230  g_uiLED1Port                     
20019234  g_uiLED2Port                     
20019238  g_uiLED3Port                     
2001923c  _lock                            
20019240  _unlock                          
2002dfb8  __stack                          
20030000  __STACK_END                      
ffffffff  __TI_pprof_out_hndl              
ffffffff  __TI_prof_data_size              
ffffffff  __TI_prof_data_start             
ffffffff  __binit__                        
ffffffff  __c_args__                       
ffffffff  binit                            
UNDEFED   __mpu_init                       
UNDEFED   _system_post_cinit               

[213 symbols]
